:1000000001242843294F4B31484D41C0D0C0E00561
:100010001BE51BB40707751B00B2B3D200D0E0D0BC
:02002000D032DC
:100023003275815511CC11FD11FD30B50553877F14
:1000330001384387803000F0C20020B30431A101AE
:100043002B200204C2B2012BD2B211731153012B24
:10005300C2ACC2B2D2997908E7B4240A3099FDC27E
:1000630099D2B2D2AC223099FDC299F59909015BBC
:1000730075082D750D0A750E0D750F2420020D756B
:10008300092D750A2D750B2D750C2D2275082075FC
:100093000920750B2E750C30E51030030575082DFE
:1000A300F404C3135003750C3575F06484B4010470
:1000B3002430F508740AC5F084B4000201C5243065
:1000C300F509E5F02430F50A22758921751B001125
:1000D300E85110310211DFC2B3C2B22275B8027502
:1000E300A892D28C22758DFD758BFD438780D28EAD
:1000F300759850C299C298C29C22C297D297223156
:1001030009311A312722D297D296C294C29522314D
:100113006422311A314922C294C29774063187C2CC
:1001230094D29722C294C2977401318774003187A5
:10013300C294D297317D22C294C29774053187311C
:1001430095C294D29722C294C29774028EF0A2F001
:1001530092E33187EF3187ED3187C294D297317DB6
:1001630022C294C29774038EF0A2F092E33187EF18
:1001730031873195FDC294D297227999313A30E093
:1001830002D9F9227808C294339295D294D8F7C24F
:1001930095227808D294C294A29633D8F7225110AC
:1001A3005117400221CC512E5129511051174002B1
:1001B30021CC512E5133E519600221CCD202E51135
:1001C300B4FF03D20322C20322C2022231D17FB77A
:1001D300DFFE227F28DFFE227F1CDFFE227F03DF7C
:0101E300FE1D
:1001E400227E08C2AFC29300D29331E0A29392E080
:1001F4000331DBD2AFDEEC227E08A2E0C2AFC293B1
:10020400929331D6D293D2AF03DEEF22C29331CF91
:10021400D293227E3C30930631E0DEF9C32231E0F2
:10022400DEFCA29322744431FC2274CC31FC22748F
:10023400BE31FC79107809751A0031E5F751490986
:10024400D8F8A71A22C0E0C0F0C0E075F008651A1B
:1002540013E51A5002641813F51AD0E003C0E0D570
:09026400F0ECD0E0D0F0D0E02273
:00000001FF
